:020000040000FA
:060000000219FD02031CC1
:03000B0002008D63
:03001300020537AC
:03001B0002009050
:03002B000202D1FD
:03005B0002054655
:030073000203097C
:100080000406080C10182030406080A0C0054032E3
:10009000C2AFC2A853E6EFC28E856B8BC0D0D2D35D
:1000A000C0E0C0F0C2CAA8CCA9CDD2CAD2AF758A6E
:1000B00000C3E8956CF8E9956DF9C3E913F9E81305
:1000C000F8E5666007C3E913F9E813F8E97025E875
:1000D000956E4020956E501CE582B410177C007B15
:1000E000007A007908900000A86AE5667004C3E809
:1000F00013F801FD900000D2A8D2AA61E7E0FDC389
:100100009CC39840EF98EB33FB0582E0FCC39DC392
:100110009840E198EB33FB0582E0FDC39CC3984017
:10012000D398EB33FB0582E0FCC39DC39840C59890
:10013000EB33FB0582E0FDC39CC39840B798EB33DB
:10014000FB0582E0FCC39DC39840A998EB33FB05F7
:1001500082E0FDC39CC398409B98EB33FB0582E093
:10016000FCC39DC398408D98EB33FB0582217890AA
:100170000000D2A8D2AA61E7E0FDC39CC39840EF7B
:1001800098EA33FA0582E0FCC39DC39840E198EAFF
:1001900033FA0582E0FDC39CC39840D398EA33FA52
:1001A0000582E0FCC39DC39840C598EA33FA0582F6
:1001B000E0FDC39CC39840B798EA33FA0582E0FC9F
:1001C000C39DC39840A998EA33FA0582E0FDC39C19
:1001D000C398409B98EA33FA0582E0FCC39DC3981C
:1001E000408D98EA33FA0582EBC46B6A54F0F9EA61
:1001F000C454F0C3996009900000D2A8D2AA61E764
:10020000EBF4C454F0F9EAF4C4540F49FAEBF4C423
:10021000540FFBC3EAF99460FAEB9400FB5020C33F
:10022000E97B007A0079006016C3135006F9C39584
:1002300052600AE9F5527553007900800205533087
:100240003A27C3EA94D0F8EB9407F9400BE8FAE9AF
:10025000FB203509D235415D303502C235203902E7
:10026000B235C3EA33FAEB33FBEB2B3B3BF9C3EB81
:1002700013FBEA13FAEA29FAEB3400FB30E3047AC1
:10028000FF7BFFE5255403601B202A18E55D33F949
:10029000EB7007C3E99A4002E9FAE53CC4332AFA55
:1002A000EB3400FBC3EA33C4540FF8EB33C454F00F
:1002B00048F87005EA60027801900000D2A8D2AA3E
:1002C000E5226002152281D4900000D2A8D2AA6152
:1002D000E7C0D0C0E0C2CF0541E5666009E56560D2
:1002E000057565006104756501E52360021523C38A
:1002F000E55460057555006104E5552401F5555038
:10030000037555FFD0E0D0D032C2AF53E67F75926F
:10031000FA7593FFC22053917FD2AF32C0E0E58AD5
:10032000303408856B8BF0A3D0E032D0E0C2AF53FD
:10033000E6EFC0D0C0E0C0F0D2D3D2AF5388EFA870
:100340008AA98CAA40308D010A758A00758C0075C7
:100350004000438810E566700AC3E833F8E933F9D2
:10036000EA33FA30331FE8C4540FFAE9C454F04AB0
:10037000FAC3132AFAC3E833F8E933F9E82AFAE9A9
:100380003406FB61D830320FC3E833E933FAE82A88
:10039000FAE93400FB61D8303115E875F056A4AAAB
:1003A000F0E975F056A42AFAC5F03400FB61D8C311
:1003B000EA13FAE913F9E813F8E875F056A4AAF07D
:1003C000E975F056A42AFAC5F03400C313FBEA130A
:1003D000FAC3EB13FBEA13FAC3EB94125009C3EA16
:1003E0009434EB940750160522E52270021522C3BF
:1003F000E52294325002A12A755400A12DE5226015
:100400000215223036067C007D088117AC31AD32F2
:10041000303A04AC33AD34C3EA9CFAEB9DFB92084E
:10042000AE60AF61303A425007203509D235813590
:10043000303502C235303504AE62AF63203902B2C6
:1004400035C3EA33FAEB33FBA208500AEAF424017D
:10045000FAEBF43400FBC3EA9450FAEB9400FB503F
:100460001478007A007B008175A208500878007A21
:10047000007B0081D4E5255403601B202A18E55D2C
:1004800033F9EB7007C3E99A4002E9FAE53CC4335B
:100490002AFAEB3400FBEA8EF0A4F9AAF0EB8EF016
:1004A000A42AFAC5F03400FBC3EB13FDEA13F8C32A
:1004B000ED13FDE813F80FEF146004C3E833F8C33D
:1004C000E933EA33FAEB33FBDFEDEB30E30678FF99
:1004D0007AFF7B078854D230E86003755500C3E586
:1004E0005BFC955C4002AC5CC3EC95545008EC7529
:1004F000F008A4FAABF0EAF4F8EBF45407F98856E4
:10050000895775230AE55A30E210D0F0D0E0D0D0F8
:1005100053F7DF43F74043E61032D0F0D0E0D0D0BD
:1005200053D8FE43DA0143E6103275230AD0F0D0E7
:10053000E0D0D043E61032C2AAD28EC2CA85CC6CBB
:1005400085CD6DD2CA32C2AFC0D0C0E0D2D38556FD
:10055000FB8557FC85575A53F7BF53DAFED2A830B4
:100560003402D2AA53E6EF53F7DF53D8FED0E0D0DF
:10057000D0D2AF327901801479038010790A800CCF
:10058000791E80087964800479C880007817E4D5E2
:10059000E0FDD8FAD9F62278FF20282879A1E76073
:1005A00023E548601F74FF8548F084853FF03029BB
:1005B0000375F005A4F8C5F0600278FFC3E8955D07
:1005C0005002A85D885C22C3E54794A0E5489400EA
:1005D000E55C500314A1D8046002F55C2275E89034
:1005E00022055EC3E55E9408405330EDF4A8BDA932
:1005F000BE755E00E9FA79A0E76041EA7006E55F42
:100600006018800CC3E8955F600EE55F5005600AD6
:100610001480070460FA8002E55FF55FC3956940C6
:100620001B755BC0C394044013755B80C394044086
:100630000B755B40C394044003755B0022E55B24AB
:1006400010500274FFF55B22743279A687F0A4C5BE
:10065000F0A2F733F55D227547007548F022C2AF6E
:10066000C2CAA8CCA9CDAA4130CF010AD2CAD2AF02
:10067000C3EA13FAE913F9E813F8AB42AC43884232
:100680008943C3E89BF8E99C20280A547FF9302C61
:1006900002E17CC1D5AD448A44F9EA9D547FFA60F9
:1006A0000678FF79FFC1BAAE45AF468B458C46A8A8
:1006B00042A943C3E89EF8E99FF9C3E54813FBE567
:1006C0004713FAE82AF547E93BF54850067547FF16
:1006D0007548FFE122AA47AB48AC47AD487E047F8E
:1006E00002C3EB9404400D1E1FC3EB940840052089
:1006F00029021E1FC3ED13FDEC13FCDEF7C3EA9CB9
:10070000FAEB9DFBEF6009C3E913F9E813F8DFF793
:10071000EA28FAEB39FB8A478B4850067BFF8B4768
:100720008B48C3EB94025002D22C3028047F03E1A3
:100730004D7892E6FFC3E53D948240110FC3E53D3D
:1007400094A040010FC3EF940640027F057E02E5AE
:1007500048C4540FF9E548C454F0F8E547C4540FB1
:1007600028F8C3E89EFAE99400FB4009C3EA940123
:10077000EB940050047A01E4FB0207C8AA47AB4897
:10078000EBC4FEEAC4540F4EFCC3EA9CFAEB94009F
:10079000FBC3E813C313F8EA28FAEB3400FB8A47DB
:1007A0008B48C3EB94024002C22C7802EBC4FE7B60
:1007B00000EAC4540F4EFAC3EA98FA4005C3940104
:1007C00050027A017892E6FF302002E1C8854E920D
:1007D000854F93D22043E680C3E49AF8E49BF9C3A3
:1007E000E833F8E933F9302C0302085DE8FAE9FB55
:1007F000D3E913FDE813FC884E894FC3EF940360DF
:1008000038EF20E00CE82CF8E93DF9ECFAEDFB803C
:1008100013E828F8E939F9C3E82401F8E93400F9C4
:100820007AFF7BFFC3EF9403400F8A508B51884AB5
:10083000894B8C4C8D4D020892885089518A4A8B85
:100840004B8C4C8D4D3028127550F07551FF754C06
:10085000F0754DFF754EF0754FFF020892E8FAD320
:10086000E813FC884EC3EF94036021EF20E007E813
:100870002CF8ECFA017DE8282401F87AFFC3EF9404
:100880000340098A50884A8C4C02089288508A4A50
:100890008C4C3020020192753A02D22043E680E56A
:1008A000255403602DA847A948C3E913F9E813F8B4
:1008B000302804E92440F9C2AF53E67F759100C3A4
:1008C000E498F594E499F595759104D22043E68077
:1008D000D2AF22D221754900752000302B0375203C
:1008E0004001F1D221754900752040302B0375205D
:1008F0000078017901202C20E52554036002C221F3
:100900007914E548C313700104F8C39414400278C5
:1009100014302804781B791BC3E833F8C3E933F992
:10092000202010E549600C302803D53A04D222215A
:10093000A4119A0549E5BF5440B52002218E302804
:100940000908C3E899400118212020210A08C3E8BA
:1009500099400201F12120C22153E67F75910030B8
:100960002C117594007595F0759104D22043E680A2
:100970000208F1E5487EFFC3334009C3334005C395
:10098000334001FEC3E49E759400F5952168C3E5EC
:10099000399401500201F130210201F1D80221A263
:1009A0002120C222C2AF53E67F7591008550948505
:1009B0005195759104854A92854B93D22043E680E8
:1009C000D2AFE52554036007202902053980103095
:1009D000220D202B0A2021071581158102141B22CC
:1009E00078003021027801E53D75F007A4F9E5F0C3
:1009F00028F5F0E9A2F013A2F113A2F213F53DC31A
:100A000094785003753D78C3E53D953E400CC29007
:100A1000C291C29275D4FF75D507302002411A8564
:100A20004C92854D93D22043E68022203817C2AFE6
:100A3000C291C285D290D29275D47F75D507D2AFBC
:100A400075AA53614FC2AFC291C287D292D290753C
:100A5000D4DF75D507D2AF75AA53614F203817C2BE
:100A6000AFC292D29175D4BF75D507C285D290D24C
:100A7000AF75AA43614FC2AFC290D29175D4BF7512
:100A8000D507C287D292D2AF75AA63614F203817BB
:100A9000C2AFC290C287D292D29175D4BF75D5072A
:100AA000D2AF75AA63614FC2AFC292C285D290D253
:100AB0009175D4BF75D507D2AF75AA43614F203861
:100AC00017C2AFC291D29075D4DF75D507C287D255
:100AD00092D2AF75AA538077C2AFC291D29275D429
:100AE0007F75D507C285D290D2AF75AA538060209A
:100AF0003817C2AFC292C286D291D29075D4DF7538
:100B0000D507D2AF75AA438046C2AFC290C286D283
:100B100091D29275D47F75D507D2AF75AA63802F15
:100B2000203817C2AFC290D29275D47F75D507C254
:100B300086D291D2AF75AA638015C2AFC292D2900D
:100B400075D4DF75D507C286D291D2AF75AA43227C
:100B50007A147B7880127A107B8C800C7A0D7BB4AF
:100B600080067A0B7BC88000E564D5E0012279021B
:100B7000E4C291D5E0FDD286D291D5E0FDC291D5F7
:100B8000E0FDC286D291D5E0FDE920E004D285D215
:100B90009030E004D287D292E564D5E0FDE920E010
:100BA00002C29030E002C2927496D5E0FDD9C1EA4B
:100BB000F8D5E0FDD8FBDBB0C29122C290C291C251
:100BC00092C290C291C29275D4FF75D507227880E7
:100BD00076FF0876FF0876FF0876FF0876FF08762E
:100BE000FF0876090876FF087601788C760108768A
:100BF000FF0876FF0876FF0876FF0876FF08760381
:100C00000876FF0876FF0876FF0876250876D00874
:100C100076280876500876040876FF08760208766B
:100C2000FF08767A0876FF0876070876010876FFCF
:100C30000876FF08760008760022FA75F00CA4AB5F
:100C4000F0EAC333F8740133F9E8C333F8E933F950
:100C5000E8C32BF8E93400F9E8C333F8E933F922A3
:100C60007888E6C39403D23A5002C23AC238E630DA
:100C7000E102D238A23892397886E6149000809347
:100C800078A6F67886E6F53FC394025003753F02D6
:100C9000789CE6753EFFB40203753EA0B40303756D
:100CA0003E8278A0E6F8600674282409D8FCF5692D
:100CB0007896E6913A88318932789EE6913A88337F
:100CC00089347897E6913A8835893671BB22303677
:100CD000117A007B007CFF7D007E00B1348B618A3D
:100CE0006022303A227896E6FA7B00789EE6FC7D18
:100CF00000C3EA33FAEB33FBC3EC33FCED33FD7E88
:100D00000AB1348B638A627896303A02789EE6FAAA
:100D10007B007897E6FC7D007E00303A10C3EA3312
:100D2000FAEB33FBC3EC33FCED33FD7E0AB1348BBD
:100D3000618A6022C3EC9EFCED9400FDC3EC9AFC3A
:100D4000ED9BFDC3EC9423ED940050047C237D00C7
:100D5000C3EC94FFED940140047CFF7D017BFF0B0D
:100D60007A000AEA7009C3EC33FCED33FDA15FECB5
:100D70008AF0A4AEF0ED8AF0A42E947C40E4EAF46C
:100D800060DD22D23691CE1205801205807A007B7A
:100D9000007C10120578E5542AFA74003BFBDCF362
:100DA0007C04C3EB13FBEA13FADCF7FFEB60027F72
:100DB000FFC23691CE2278A5E6F95403D2837002A1
:100DC000C283E9540CD2847002C284E954307000AA
:100DD000E954C07000227567007568007597DE756C
:100DE00097AD7581C043FF8075EF0675A90071BB93
:100DF00075800275F1FF75A4F875800275D4FF75D2
:100E0000900075F20775A50775900075D50775A652
:100E10000175E34075E20271BBE4F8F6D8FD71CECE
:100E200012146578988664753001C2AF1205887116
:100E3000501205807156120580715C120580B1B6A2
:100E4000C2AF75670075680078FA79FA308107D902
:100E5000FBD8F7021C00916091CE7898866471BB34
:100E600075A91375A71075C10075A7007566007583
:100E7000E401758811758E0475890975C80475912A
:100E80000475D84075D90875F783759E007596026C
:100E900075DA4A75DB0075A82375E69075B801759B
:100EA000BF8075AB0075D10C75BCB975BB1075E80A
:100EB0008075B201120574D2AF753C00C2301205C4
:100EC00088C231C232C233C23475520075530075C4
:100ED0002200120584C3E522940A5002E1A6D23111
:100EE000752200120584C3E522940A5002E1A6C2CD
:100EF00031D232752200120584C3E522940A5002D1
:100F0000E1A675E491758851758E017589AA758C75
:100F100000758D00C2A9D2ABD2AA756B80756A1418
:100F2000756E50C232D23475220A120584756A1069
:100F3000C3E522940A7552007553004069758E0C02
:100F4000756B00756A28756E2875220A12058475FE
:100F50006A20C3E522940A75520075530040477514
:100F60008E0C756B80756A14756E1475220A1205E5
:100F700084756A10C3E522940A75520075530040C7
:100F80002575E401758811758E04758909D2A9C289
:100F9000ABC2AAC234D233752200120584C3E52243
:100FA000940A4002C140120578203003020E40C26C
:100FB000AF715071507150D2AF1205882034033098
:100FC0003A0302106B120578788CE6C39401500343
:100FD00002106BE530C39401500302106B7567A5D6
:100FE0007568F17F02D23691CE120584C2AFC23647
:100FF00091CEC3E554947FD2AF4070120574C2AF56
:10100000120B62D2AFDFDE120D83C3EF7897F612B8
:101010000588B1527F0AD236120CCE120584C2AFB7
:10102000C236120CCEC3E554947FD2AF50E61205FF
:1010300074C2AF120B5012057C120B50D2AFDFD628
:10104000120D83EF24037896F6F87997E7C394237B
:101050004003985006E824237897F612058891AC4F
:10106000B181120584120CCE020E407567007568BE
:1010700000120584C3E55494014003020FBCC2AFC3
:10108000120B62120B62120B62D2AF12058875301E
:1010900000E4F537F5380537E537F4703F05387863
:1010A0009AE67819146012783214600D787D146015
:1010B0000878FA146003753800C3E53898401D12AB
:1010C0000BBB120574153875370078998664C2AF6A
:1010D000120B62D2AF7898866412058412057CE503
:1010E000237003020E40C3E5549401500AC3E55235
:1010F00094015016021096120584E5237003020E27
:10110000407552007553000212ACC3E55294017051
:1011100017C2AF120BBB78998664120B5078988671
:1011200064D2AF120584419EC3E55294027017C287
:10113000AF120BBB78998664120B5678988664D2EE
:10114000AF120584419EC3E55294037017C2AF12DB
:101150000BBB78998664120B5C78988664D2AF12C8
:101160000584419EC3E55294047017C2AF120BBBB5
:1011700078998664120B6278988664D2AF120584DF
:10118000419EC3E55294057017C2AF120BBB78990C
:101190008664120B6278988664D2AF120584419EF1
:1011A000C3E55294077019C3E5539406500201E653
:1011B0007401303A0274037888F6C238C239419E0D
:1011C000C3E55294087019C3E5539406500201E632
:1011D0007402303A0274047888F6D238D239419ECB
:1011E000C3E55294097017C3E5539406500201E613
:1011F000303A0BC37888E69402F6C23A419EC3E5C2
:1012000052940A7016C3E5539406500201E6203A40
:101210000A7888E62402F6D23A419EC3E552941435
:101220007025C3E5539406500201E6C2AF901A0B35
:10123000740093D2AF7888F613C238C2394002D214
:10124000384002D2398057C3E55294157038C3E54F
:10125000539406404FC2AF901A0B740093D2AFF86C
:10126000B801027402B802027401B803027404B82F
:10127000040274037888F613C238C2394002D238A7
:101280004002D2398018C3E552940C70117567A5DD
:101290007568F1C3E5539406400A91ACD2AF75521C
:1012A0000075530075670075680001E6C2AF120B48
:1012B000BBE4D2AFE4F55EF524F525F53D755E0897
:1012C0001205741205DD30EDFDA8BDA9BEE970015F
:1012D000F8885F1205E1755E08C2AF120648855DA9
:1012E0005B855D5CD2AF75A71075C13075A70075C1
:1012F000A903756601303A07C238303502D238D2B8
:1013000028753900120AEF120B2012065712065EDA
:1013100012065712065E1206571208E31209E0126F
:101320000A2B12065E1208D3202C03120597302CCC
:10133000031205C71209E0120A5C12065E1208E3E6
:101340001209E0120A8D12065E1208D31209E01289
:101350000ABE12065E1208E31209E0120AEF120634
:101360005E1205DD1208D31209E0120B201205E10E
:1013700012065E302827855D5B79187A0CC3E53943
:1013800099400EC228D2298A3B855D5B855D5C80D1
:101390000CC3E55494014003021319812330291F23
:1013A000202B1CE53B147006C229D22A6119F53B9B
:1013B000203A07C3E5549401400302131980647571
:1013C0003C00203A0F78FA79A4E760027803C3E57D
:1013D0005598504FE523604B303A1720380520359B
:1013E00007800F303502800A202B07D22B855D5BEA
:1013F000614978F0302B05855D5B7820C3E548981E
:101400005003021319302B1BC22BC238303502D2C5
:1014100038D229753B12855D5B6119053CE5546046
:10142000028126753C00C2AF120BBB7524007525E6
:101430000075A91375A71075C10075A70075660022
:10144000D2AF120584120BBB78A4E6600CC285D221
:1014500090C286D291C287D292C3E53C94044003E5
:10146000020E400191901A0D782091E5E520B455C7
:101470000AA391E5E520B4AA0280137567A57568F3
:10148000F1120BCE91AC756700756800801D901A43
:101490000378807B0A91E5A308DBFA901A0F788C19
:1014A0007B1A91E5A308DBFA901A2922C2AFB12872
:1014B000B105901A00741091EAA3740791EAA3741D
:1014C0002191EA901A0378807B0A91E9A308DBFA5C
:1014D000901A0F788C7B1A91E9A308DBFAB13BB123
:1014E00019901A2922E493F622E6438F01538FFDC7
:1014F000FFC3E583941C400122EF8567B78568B779
:10150000F0538FFE22438F02438F018567B78568B2
:10151000B7901A0DF0538FFC22901A0D745591EA72
:10152000901A0E74AA91EA227A3079D07820901A13
:101530004091E5E520F709A3DAF7227A3079D090D7
:101540001A40E791EA09A3DAF9227C05120588DC42
:10155000FB22C2AF120B50120B56120B5C120B6225
:1015600012057C120B50120B56120B5C120B6212FE
:10157000057C120B50120B56120B5C120B62D2AF91
:1015800022C2AF120B62120B5C120B56120B5012DE
:10159000057C120B62120B5C120B56120B501205DB
:1015A0007C120B62120B5C120B56120B50D2AF2244
:1019FD00020DD6100721FFFFFFFFFFFF09FF01FFBB
:101A0D0055AA01FFFFFFFFFF03FFFFFF25D0285061
:0D1A1D0004FF02FF7AFF0701FFFF0000FF3A
:101A400023515F485F303023202020202020202099
:101A500023424C48454C492445464D3842323123B7
:101A60002020202020202020202020202020202076
:101C0000C2AFC2D37597DE7597AD7581C075A90057
:101C100043FF80752438752503B1DB7529A5752A26
:101C2000F143F10253A4FDD28175D4FF75E3407DE9
:101C3000FA780379E67C10752200752300901DE880
:101C40007B06752498752501308102814820810822
:101C5000D8FBD9F9DCF781BA308108D8FBD9F9DC97
:101C6000F781BAB19BE493A3C39A6004DDC381BA40
:101C7000DBDBB18D600281317B08E493FAA3B16EA6
:101C8000DBF87A30B16E752200752300B18DEAFC65
:101C9000EBFDC3ED94FE400EB18D8A278B28ED300D
:101CA000E0048A828B83B18D7AC270D8C3ED94FE32
:101CB000601950CEBD0029EC600F7520007521FF22
:101CC000752900752A000200008100A827A92808AC
:101CD00009D804D90281DDB191EAF281D10D81A642
:101CE000C3ED94035051EDA2E092007AC5C3E582A2
:101CF0009400E583941C508C200010438F02438F86
:101D0000018529B7852AB7F0300027A827A9280818
:101D100009438F01538FFDD804D902A132C3E58353
:101D2000941C4003A3A117E28529B7852AB7F0A325
:101D3000A117538FFC81827AC1BD030CE493A3FAEF
:101D4000B152DCF8B14A81828184AA22AB23B16E00
:101D5000EBFAEA6222752608C3E52313F523E52290
:101D600013F52250066323A0632201D526EAB1DBD6
:101D7000B1DB75260AEAF4200102D281300102C2E9
:101D800081B1DBC3134002C201D526EB22B191EA37
:101D9000FB208102A191308102A196752608AE2414
:101DA000AF25C3EF13FFEE13FEB1DFB1DBC3EA13C0
:101DB0003081024480FA30E703632201C3E5231334
:101DC000F523E52213F52250066323A0632201D5F3
:101DD00026D9E52265236523F52222AE24AF250E00
:101DE0000FDEFEDFFCD20122424C48656C693437BD
:061DF0003164E8B20601B7
:00000001FF
